S111C000546869732070726F6772616D2069F5
S111C00E7320636F707972696768742031392A
S111C01C3934202062793A2020202020202070
S111C02A20202020202020204772616E7420E8
S111C0384265617474696520202045646D6F53
S111C0466E746F6E2C2020414220202020209A
S111C0542043616E61646120202020202D2D88
S111C0622D2D2D2D2D2D2D2D2D2D2D2D2D2D56
S111C070416C6C207269676874732020202074
S111C07E20207265736572766564212020545B
S111C08C6869732070726F6772616D206D6158
S111C09A79206E6F7420626520636F70696593
S111C0A864206F722020202075736564206967
S111C0B66E2077686F6C65206F72696E207063
S111C0C461727420776974686F7574207468F3
S111C0D26520657870726573736564202020A4
S111C0E07772697474656E20636F6E73656E9B
S111C0EE74206F662074686520617574686F35
S111C0FC722E202043616C6C49442C20566542
S111C10A7220312E303300313939342C204765
S111C1182E2042656174746965002A20496E08
S111C126697469616C697A696E67202A002A5F
S111C134202020204E616D65732120202020E4
S111C1422A002A2057616974696E6720666FAF
S111C1507220202A002A20202063616C6C20BB
S111C15E2E2E2E2020202A0043686F6F73655A
S111C16C204E616D653A20230021202042619F
S111C17A6420204550524F4D202021002120EA
S111C18843616C6C20466163746F72792021F0
S111C1960012151515151512008640B7103944
S111C1A48E00FFBDCD508638B74000BDCD5093
S111C1B28601B74000BDCD50860FB74000BDDA
S110C1C0CD508606B740008640BDCD50B777
S111C1CD4000C608CEC197A60008BDCD365A64
S111C1DB26F78601BDCD50B74000BDCD561AE3
S111C1E983A3BD2716CEC175BDCD3F86C0BD54
S111C1F7CD50B74000CEC186BDCD3F20FECE58
S111C205C100BDCD3F86C0BDCD50B74000CEB8
S111C213C111BDCD3FCE00C8BDCCB20926FA84
S111C2218601BDCD50B74000CEC122BDCD3F39
S111C22F86C0BDCD50B74000CEC133BDCD3F5B
S111C23DCEB610C607A6008130240A8630BD96
S111C24BCCBFBDCCD4200C813923088630BD75
S111C259CCBFBDCCD4085A26E0C610A6008186
S111C26720240A8620BDCCBFBDCCD4200C817F
S111C2757F23088620BDCCBFBDCCD4085A263A
S111C283E0A60027074FBDCCBFBDCCD4088C6D
S111C291B7F025AB8606B7102B4FB7102C86DE
S10EC29F04B7102D4F97049705970C6F
S10DC2AA970ECE000FDF08860197FF
S10EC2B4028600970D860197064FB725
S111C2BF10268640B710240EB6102E842026BA
S110C2CD037EC669B6102FD60DC1162303DB
S111C2DA7EC39958CEC2E63AEE006E00C3143D
S109C2E8C331C373C3BCA3
S109C2EEC3F3C422C4479F
S109C2F4C470C484C49967
S109C2FAC4C8C4F0C569CC
S109C300C590C5C4C5E0B0
S109C306C399C399C39919
S109C30CC399C609C61E18
S10FC312C64081042609970A8601970D95
S110C31E7EC669818027037EC669970A8662
S10FC32B07970D7EC6698109260D97074F
S10CC3379B0A970A8602970D7E09
S110C340C358811227078600970D7EC66939
S10CC34D97079B0A970A8603B7BF
S10FC356000D9604810A25127A0004CE22
S110C362000FC6BDA615A700085A26F8DF77
S110C36F087EC669813025228139221EDE38
S10CC37C08A70008DF089B0A97DA
S10EC3850A7A00079607810127037E57
S10FC390C6698604970D7EC66986009776
S10FC39C0DCE000F96042706C6153A4A81
S10FC3A826FCDF087D000C2604C601D72B
S109C3B402960497057EC9
S110C3BAC669813025308139222CDE08A7A8
S10CC3C70008DF089B0A970A7ABA
S110C3D000079607810A27037EC6698605CB
S10FC3DD970DDE088603A70008860AA757
S110C3E90008DF087EC6697EC399814F27D6
S110C3F607815027037EC399DE08C604E7C3
S110C4030008C601E70008A70008DF089B39
S10CC4100A970A7A000727037E4B
S110C419C3998606970D7EC6698130251EE5
S10FC4268139221ADE08A70008DF089BF9
S10CC4320A970A7A000727037E29
S10DC43BC6698606970D7EC6697E69
S10FC445C3999B0A27037EC399860097C5
S10EC4510D7D000C2604C601D70296E6
S10AC45C044C97049705CE80
S110C463000FC6153A4A26FCDF087EC669A4
S10FC470810D24037EC399970B9B0A974F
S10FC47C0A8608970D7EC669810127031B
S10BC4887EC3999B0A970A7A0E
S110C490000B8609970D7EC66981082703FD
S10CC49D7EC39997077A000B9BFA
S10BC4A60A970A860A970D9615
S110C4AE04810A25127A0004CE000FC6BDD9
S110C4BBA615A700085A26F8DF087EC669FA
S110C4C8813025218139221DDE08A70008DE
S10AC4D5DF089B0A970A7AB5
S110C4DC000B7A000727037EC669860B97C4
S110C4E90D7EC6697EC3998103271381046B
S111C4F62724810627358107273F8108275018
S10EC5047EC399DE08A70008DF089B37
S10CC50F0A970A7A000B860C97C6
S10DC5180D7EC669DE08A70008DFE7
S109C522089B0A970A7A47
S10DC528000B860E970D7EC6699B7A
S10CC5320A970A7A000B8614979B
S10DC53B0D7EC669DE08A70008DFC4
S109C545089B0A970A7A24
S10DC54B000B8610970D7EC669DE12
S10CC55508A70008DF089B0A97FF
S10CC55E0A7A000B8612970D7E87
S111C567C6698107270B81082707810B27036C
S10EC5757EC399DE08A70008DF0897CA
S10AC580077A000B9B0A97E8
S110C5870A860DB7000D7EC6698130252D92
S10FC59481392229DE08A70008DF089B7B
S10AC5A00A970A7A000B7AE6
S111C5A7000727037EC6697D000B2607861653
S10DC5B5970D7EC669860B970D7E74
S110C5BFC6697EC399810127037EC399DEFE
S10CC5CC08A70008DF089B0A9788
S10CC5D50A7A000B860F970D7E13
S111C5DEC669814F2707815027037EC399DE6B
S10CC5EC08A70008DF089B0A9768
S10EC5F50A7A000B26078616970D7EBD
S110C600C669860B970D7EC669810127036C
S10BC60D7EC3999B0A970A7A87
S110C615000B8615970D7EC669814C270722
S10FC622815227037EC3999B0A970A7A71
S110C62E000B26078616970D7EC669860B45
S10DC63B970D7EC6699B0A27037E53
S110C645C3998600970D7D000C2604C601E4
S10BC652D70296044C970497EB
S10FC65A05CE000FC6153A4A26FCDF0886
S10FC6667EC6697D000C27037EC6EB7DB8
S110C672000126037EC6EB7D0002266DB696
S110C67F1008840426099605810123604AF1
S110C68C2010B610088402261796054C9164
S10EC699042302204D97058601970240
S111C6A47F00007F0001203F7D0003273AB68F
S111C6B21008841026070F7F00037EC19FB678
S10FC6C01008842026088601970C9702BD
S111C6CC2013B61008840826167D00042711DA
S10DC6DA9605BDCA20860197027F71
S110C6E400017F000320007D000C26447D32
S111C6F10002273F7D000426298601BDCD509E
S111C6FFB74000860CBDCD50B74000CEC144FC
S111C70DBDCD3F86C0BDCD50B74000CEC15556
S111C71BBDCD3F7F000220117F0002860CBDC1
S10FC729CD50B74000BDCB4ABDCA5E969F
S110C7350C810126697D000226647D00014F
S110C742275FB610088402260996064C8174
S110C74F142312204FB610088404261796F8
S10FC75C064A81012402203F9706860152
S10EC76897027F00017F000020317D5C
S111C77300032717B610088420261086FF97AF
S10CC7810C860197027F00017F80
S111C78A00032015B610088418260E860297A8
S10CC7980C860197027F00017F69
S110C7A10003960C8101263F7D0002273A1B
S111C7AE8601BDCD50B74000CEC166BDCD3F63
S10CC7BC9606BDCD15BDCCECBD03
S111C7C5CD3617BDCD3686C0BDCD50B7400071
S110C7D3CEB617C61896064A27033A20FA78
S110C7E0BDCD3F7F00022000960C81FF2795
S110C7ED037EC88D7D000227037EC88D7D6C
S111C7FA000126037EC88DB6100884022606B0
S111C808B640014C200BB6100884042644B63A
S111C81640014AC610BDCD50F74000F6400068
S111C824C440260E8130240286398139231047
S111C8328630200C81202402867F817F230221
S111C8408620BDCD50B74001C610BDCD50F7C7
S10FC84E40007F0001863297002034B6C1
S111C85A100884082605BDC9E920EB7D000303
S111C8682723B6100884102607BDCC0B8601CA
S110C8762008B610088420260E4F970C4CA5
S10EC88397027F00017F000320009655
S10FC88E0C81FF2658960227547F0002FC
S111C89A8601BDCD50B740008623BDCD369635
S10BC8A806BDCD15BDCCECBDAD
S111C8B0CD3617BDCD368620BDCD368620BDD3
S110C8BECD36CEB610C61896064A27033AAA
S111C8CB20FABDCAF886C0BDCD50B74000BDEE
S110C8D9CD3F8685BDCD50B74000860EBD15
S10FC8E6CD50B74000960C8102267096DD
S10FC8F202276C7F00028601BDCD50B708
S10FC8FE4000D60E4F8F960EBDCCECBD52
S111C90ACD3617BDCD36863ABDCD36C60437C0
S111C9188620BDCD36A60008BDCCECBDCD36C4
S111C92617BDCD36335A26E986C0BDCD50B7B5
S110C93440003C3332BDCCECBDCD3617BD08
S110C941CD36863ABDCD36C604378620BDFE
S110C94ECD36A60008BDCCECBDCD3617BD1E
S110C95BCD36335A26E9960C8102264A7D1A
S111C968000226457D00012740B61008840217
S110C9762606960E8B08200BB610088404CC
S10EC9832612960E8008970E8601977E
S10DC98E027F00017F0000201A7DE3
S111C99800032715B610088420260E8600978B
S10CC9A60C860197027F00017F59
S110C9AF0003B61008843E813E260C96035A
S110C9BC8105220B8B019703200A7F0003E5
S111C9C920058601B700013E7EC2C78640B736
S110C9D7102596008B01816426054FC601D2
S10EC9E4D70197003B8614BDCD50B76F
S111C9EF4000BDCD50B64000847F810826096B
S111C9FD8614BDCD50B7400039810D26098641
S111CA0BC0BDCD50B740003981502608868545
S110CA19BDCD50B7400039B1000426107A9D
S10FCA2600047A0005FC0008830015FDE4
S111CA32000839C615CE000F4A27033A20FA31
S111CA40F60004F0000586153DA615A70008B3
S110CA4E5A26F87A0004FC0008830015FD48
S111CA5B000839A6008103272481042701392D
S110CA69C6C0BDCD50F740000808A600CEA1
S111CA76CB28814F2708CECB398150270139B8
S111CA84BDCD3F39083C1838E60008C0073A1B
S111CA92BDCC758C0000270C86C0BDCD50B7FE
S111CAA04000BDCD3F39183C3886C4E600C1C5
S111CAAE07270E8001C10827088001C10A274E
S111CABC028001BDCD50B74000E60008C10A5B
S111CACA2715C10722022026A60008BDCD367E
S110CAD8862DBDCD36C1082317A60008BD6C
S111CAE5CD36A60008BDCD36A60008BDCD3660
S111CAF3862DBDCD36A60008BDCD36A60008A2
S111CB01BDCD36A60008BDCD36862DBDCD3681
S111CB0FA60008BDCD36A60008BDCD36A60092
S111CB1D08BDCD36A60008BDCD36392A204FFE
S111CB2B7574206F662052616E6765202A00C3
S111CB39204E756D62657220507269766174CB
S111CB476521008601BDCD50B740008623BD98
S111CB55CD36B600058B30813A26028600BD2F
S10ECB63CD368620BDCD36BDCD36CECC
S111CB6E000FB60005C6154A27033A20FAA6A2
S111CB7C0008BDCD36A60008BDCD36862FBDFF
S111CB8ACD36A60008BDCD36A60008BDCD36BA
S111CB988620BDCD36E60058585858A60180B8
S111CBA6301B8112242CA6000881302703BD09
S111CBB4CD36A60008BDCD36863ABDCD36A6D8
S111CBC20008BDCD36A60008BDCD368661BD87
S111CBD0CD36866DBDCD3639811227038B8894
S110CBDE19BDCCEC81302703BDCD3617BD49
S110CBEBCD360808863ABDCD36A60008BD3B
S111CBF8CD36A60008BDCD368670BDCD36867E
S111CC066DBDCD36390F8685BDCD50B74000CB
S110CC14CEB610C61896064A27033A20FA39
S110CC21C603BDCD50B64001A1002706BDDD
S111CC2ECCBFBDCCD4085A26EC8689BDCD50AF
S111CC3CB74000C604BDCD50B64001A100278C
S111CC4A06BDCCBFBDCCD4085A26EC86C0BDB6
S111CC58CD50B74000C610BDCD50B64001A16E
S111CC66002706BDCCBFBDCCD4085A26EC0E68
S111CC7439183C3736F6B61018CEB6105D27C8
S111CC8227373C183CC607A60018A100260F51
S111CC900818085A26F338C6073A1838332015
S110CC9E0E1838C618183A38335A26D9CE65
S111CCAB00003233183839183C18CE06DA1857
S111CCB90926FC183839368616B7103BA7003A
S111CCC74CB7103BBDCCB24FB7103B323936E0
S111CCD58602B7103B3236A7008603B7103B29
S111CCE3BDCCB24FB7103B32393C36CECD0536
S111CCF116545454543AE60017CECD0533C4FD
S111CCFF0F3AE60038393031323334353637E7
S111CD0D3839414243444546373C16CECD21C9
S111CD1B3AA600383339000102030405060766
S111CD29080910111213141516171819207D7D
S111CD3740002BFBB7400139A600084D260131
S111CD45397D40002BFBB7400120EF7D4000FC
S111CD532BFB39CEC00018CEC19E18FF00087D
S110CD6118CECDC1CC0000FD00058601B741
S111CD6E0007A600B4000727028601F600069F
S111CD7CC47F183C183A18E6001838F7000473
S110CD8AB80004F60005595959F70004B823
S10DCD9700044479000679000574D5
S111CDA1000725098601B10007270920C28674
S111CDAF80B7000720BBBC000827030820B390
S111CDBDFC0005390000010100000101010124
S111CDCB000001010000000001010000010150
S111CDD9010100000101000001010000010140
S111CDE7000000000101000001010101000034
S111CDF5010100000000010100000101000026
S111CE03010100000101010100000101000015
S111CE11000001010000010101010000010107
S111CE1F0000010100000101000000000101FB
S111CE2D0000010101010000010100000000ED
S109CE3B010100000101E9
S109FFD6C19FC19FC19F01
S109FFDCC19FC19FC19FFB
S109FFE2C19FC19FC19FF5
S109FFE8C19FC19FC19FEF
S109FFEEC19FC9D4C19FAC
S109FFF4C19FC19FC19FE3
S109FFFAC19FC19FC19FDD
S9030000FC
